:04000000B6017929A3
:10000800080098181812181664008C1E08281A0878
:1000180003147429040864000C1E0F2899000314A3
:100028007429B616B61EB612B6191E28B6156D2056
:1000380003185B280830A3008120A20DA30B2028F9
:10004800B61E66208B208720B61A5B206020220807
:10005800031074293617361F3613A4002908031D08
:100068003828361B5B287429251883172408840030
:1000780000088313462003187429A40AA903322808
:10008800B616B61EB61236194E28FE39B700361502
:1000980003107429361A5628A60036166D20031840
:1000A8005B282608742003185B28B61E742966206E
:1000B8008B2036113612B6113A0884003808841796
:1000C80080046C283A088400380980058417800564
:1000D800080060208B20662087203708B619013871
:1000E800A2000830A300A20D03186020031C66209C
:1000F8008B208720A30B772860208B203A08840068
:1001080038080005FF3E3B088400390969283B0888
:10011800840039086328A4002908031974296F2169
:10012800A000251883172408840020088000831362
:10013800A40AA9039028B71329080319B71704308C
:10014800A800250EAC202508AC20240EAC202408DD
:100158000F39F63E0318073E0A3EB228A000A8034E
:100168000319B71329080319BC2828020318080023
:100178002008031DB713B71B0800303E6F2908304D
:10018800A600A7003B088400390837191021371D3D
:1001980012213A08840038081521A001A101260877
:1001A80003197429B71807213A088400000838058C
:1001B800FF3EA00DA10DB71C0721A60BD6282708C6
:1001C80037183E29200874290830A6003B08840007
:1001D800390837191021371D12213A0884003809C7
:1001E800192126080319742937183E213A08840072
:1001F800A10CA00C00083804031C38068000072155
:10020800A60BFA2874293B088400390880060000E8
:100218000D290E298006080080041829FF3A800558
:100228001929841780047429FF3A841780057429D2
:10023800A301A200FF30A207031CA307031C742913
:100248000330A100E4302A211E29A101F63EA000B6
:10025800A109031C3529FE300000A0070318302926
:10026800A0076400A10F2F29000020183B2920189F
:100278003D290800A201A3014529A10CA00CA20D4B
:10028800A30DFF3E031841292308A1002208A0005E
:1002980074290310A00DA10DFF3E03184D29200855
:1002A8007429A101A301A20001305F29A101A301C2
:1002B800A20004305F29A80023082102031D662933
:1002C80022082002043003180130031902302805DF
:1002D800031DFF307429840031088A003008820029
:1002E80083130313831264000800831607309900F0
:1002F80020309800831290309800831607309F00B2
:100308000714871007118712C901C3018312FC0162
:10031800FD010130A300F4308A011D2153308A0108
:100328000F2074308A010F2061308A010F2072304B
:100338008A010F2074308A010F200A308A010F20A9
:100348000D308A010F208A110A12612D8716831633
:10035800FF30C1000A30BF0083128A110A126724D5
:10036800871232308A011C2183164030BE00953036
:10037800C000831283163E08C10007308312BA00FA
:100388000430B8000730BB000230B9000130B700B4
:10039800831641088312A000A1018A01E820831670
:1003A800C1010430BF0083128A110A126724831620
:1003B8004008C10007308312BA000430B800073083
:1003C800BB000230B9000130B70083164108831220
:1003D800A000A1018A01E82083160130BD00831224
:1003E8008A110A126B22871632308A011C21871261
:1003F800640083164A08003C8A110A128312031902
:10040800482A87168316FF30C10007308312BA00C6
:100418000430B8000730BB000230B9000130B70023
:10042800831641088312A000A1018A01E8208A11DD
:100438000A12E324871283164130C1000730831261
:10044800BA000430B8000730BB000230B9000130F0
:10045800B700831641088312A000A1018A01E82091
:100468008316C1010430BF0083128A110A1267245F
:100478008316FF30C10083128A110A12C0248A1120
:100488000A12E3248A01FC298316FF30C10049308F
:1004980083128A010F204E308A010F2049308A01C9
:1004A8000F2054308A010F2020308A010F204F304E
:1004B8008A010F204B308A010F2021308A010F203A
:1004C8000A308A010F200D308A010F2008006400CD
:1004D80083164A083D028A110A1283120319842AD4
:1004E8000730BA000130B8000730BB000230B9004D
:1004F800B7018A01C3208316CA0083128A016B2AB6
:10050800080087168316FF30BA0083128A110A1270
:10051800D1248A110A12E324871283165830B600B0
:1005280083127F088316B70083127E088316B800EB
:100538002B08B9002A08BA0083128A110A128D24DE
:100548008316FF30BA0083128A110A12D1248A1145
:100558000A12E3248316BD0183128A016B228316D3
:10056800FE30BA0083128A110A12D12483162E088B
:100578008312FC0083162F088312FD007C08A0005C
:100588007D08A100831631088312A3008316300862
:1005980083128A0157218A110A12031D012B073081
:1005A800BA001030B8000730BB000830B900A030DE
:1005B8008A0146207D088A0146207C088A01462057
:1005C8008A0115208316C10007308312BA0004304F
:1005D800B8000730BB000230B9000130B7008316FD
:1005E80041088312A000A1018A01E820FC0A03192E
:1005F800FD0A8A110A12031DC22A8316FF30C100A0
:100608000230BF0083128A110A1267248A110A1263
:10061800E3240F3083164A05CC0083128A110A128C
:10062800E324640083164A08003C8A110A128312E4
:10063800031D2E2B0730BA000130B8000730BB006D
:100648000230B900B7018A01C3208316CA00831299
:100658008A01152B8A110A1221240800871683168D
:10066800FF30BA0083128A110A12D1248A110A12A1
:10067800E324871283165130B60083127F0883164D
:10068800B70083127E088316B8002B08B9002A0821
:10069800BA0083128A110A128D248316FF30BA0019
:1006A80083128A110A12D1248A110A12E3248316AA
:1006B800BD0183128A016B228316FE30BD008312AE
:1006C8008A016B2283162E08AC002F08AD00831216
:1006D80083162C088312A00083162D088312A1000C
:1006E800831631088312A3008316300883128A0107
:1006F80057218A110A12031DB52B0730BA000130A1
:10070800B8000730BB000230B900B7018A01C32026
:100718008316C10007308312BA001030B8000730C2
:10072800BB000830B900A0308A01462083162D0886
:1007380083128A01462083162C0883128A014620D8
:100748008316410883128A01442005308A011C213E
:100758008316AC0A0319AD0A8A110A128312031D03
:100768006C2B8A110A12E3248A110A12E3248A11D3
:100778000A122124080083165030BE00FF30C00042
:1007880083128A110A12E623080083166030BE001D
:1007980083128A110A12E623080083166130BE000C
:1007A80083128A110A12E623080083160130C30057
:1007B8006630BE0083128A110A12E6238316C3012B
:1007C8008312080087168316FF30BA0083128A1135
:1007D8000A12D1248A110A12E324871283163E08CA
:1007E800B60083127F088316B70083127E0883162B
:1007F800B8002B08B9002A08BA0083128A110A1215
:100808008D248316FF30C1000230BF0083128A1185
:100818000A1267248A110A12E32464008316430823
:10082800013C8A110A128312031D1B2C080083162F
:10083800BD0183128A016B22080087168316FF30D8
:10084800C10007308312BA000430B8000730BB007B
:100858000230B9000130B700831641088312A000A6
:10086800A1018A01E8208A110A12E324871283165B
:100878004D30BA0083128A110A12D1248316C1019D
:100888000430BF0083128A110A1267248316FF30CE
:10089800BA0083128A110A12D1240730BA00013033
:1008A800B8000730BB000230B900B70110308A0128
:1008B800C4208316B200831221088316B3003208BD
:1008C800C9008312080083160130CC00831264002B
:1008D80083164C083F028A110A128312031C8C2CBF
:1008E8000730BA000430B8000730BB000230B90046
:1008F8000130B700831641088312A000A1018A01C4
:10090800E8208316CC0A8A110A128312031D6B2C65
:1009180008000730BA000430B8000730BB000230C6
:10092800B9000130B700831636088312A000A10170
:100938008A01E8200730BA000430B8000730BB004D
:100948000230B9000130B700831637088312A000BF
:10095800A1018A01E8200730BA000430B800073046
:10096800BB000230B9000130B70083163808831283
:10097800A000A1018A01E8200730BA000430B800BD
:100988000730BB000230B9000130B70083163908C0
:100998008312A000A1018A01E8200730BA000430C0
:1009A800B8000730BB000230B9000130B700831629
:1009B8003A088312A000A1018A01E8200800073044
:1009C800BA000130B8000730BB000230B900B701E7
:1009D8008A01C3208316CA008312080044308A01A2
:1009E8000F2061308A010F2074308A010F20613096
:1009F8008A010F2020308A010F2066308A010F20DB
:100A080072308A010F206F308A010F206D308A0101
:100A18000F2020308A010F204D308A010F204D30E1
:100A28008A010F2043308A010F200A308A010F20E3
:100A38000D308A010F2083162E08AC002F08AD0058
:100A4800831283162C088312A00083162D088312A4
:100A5800A100831631088312A3008316300883127D
:100A68008A0157218A110A12031D602D0730BA0026
:100A78001030B8000730BB000830B900A0308A0138
:100A8800462083162D0883128A01462083162C08D7
:100A980083128A0146208A0115208316C100410865
:100AA80083128A010F208316AC0A0319AD0A8A1132
:100AB8000A128312031D252D08008A01AA21FE01AE
:100AC800FF018316AA010230AB0083128A01BF23FB
:100AD8008316AE01AF01FF30B0000130B1008312C0
:100AE8008A110A12772D57308A010F2061308A0146
:100AF8000F2069308A010F2074308A010F20693075
:100B08008A010F206E308A010F2067308A010F207A
:100B18002E308A010F202E308A010F200A308A01D8
:100B28000F200D308A010F2011308A010F2011305B
:100B38008A010F2011308A010F208A010520403CCC
:100B48008A110A12031DA12D0B30A9000530B0002F
:100B5800B101A501A0308A018F2013308A010F202E
:100B680013308A010F208316C601831264000B30EC
:100B7800831646028A110A1283120318022E83165C
:100B88004608A03E840000088312B200FF30A2008D
:100B9800A20A22080F3C8A110A12031CF62D8A1198
:100BA8000A12E22532028A110A12031DCC2D2208EC
:100BB8008316C40083128A110A12F62D05308A00A2
:100BC8002208820730343134323433343434353403
:100BD8003634373438343934413442344334443485
:100BE8004534463483164608A03E840044088000F5
:100BF800C60A8A110A128312031DBA2D8316200809
:100C0800C80021088312A000A10104308A015021E4
:100C1800B2002108B3008316220883123204831617
:100C2800BB0023088312A000A10104308A015021CF
:100C3800B2002108B3008316240883123204FF008F
:100C4800831625088312A000A10104308A015021CF
:100C5800B2002108B3008316260883123204FE006E
:100C6800831627088312A000A10104308A015021AD
:100C7800B2002108B30083162808831232048316B1
:100C8800AB0029088312A000A10104308A01502179
:100C9800B2002108B30032088316AA0464003B0896
:100CA800003C8A110A128312031D5E2E831601303E
:100CB800BB008312640083164808003C8A110A129C
:100CC800831203198D2E640083164808013C8A118B
:100CD8000A12831203193A2F640083164808023C4B
:100CE8008A150A1283120319062864008316480815
:100CF800033C8A150A1283120319A8286400831674
:100D08004808043C8A150A1283120319AA288A0182
:100D1800982D11308A010F2041308A010F2064304C
:100D28008A010F2064308A010F2072308A010F2057
:100D38003A308A010F200430A9007E08A4007F08F9
:100D4800A5000E30B000B1018A019F200430A9002F
:100D580083162A088312A40083162B088312A50081
:100D68000E30B000B1018A019F200A308A010F209D
:100D78000D308A010F2013308A010F2083160130AD
:100D8800BC008312640083163C083B028A110A12D5
:100D98008312031C382F8A01322383162E08AC00D5
:100DA8002F08AD00831283162C088312A000831627
:100DB8002D088312A100831631088312A30083161D
:100DC800300883128A0157218A110A12031D212F24
:100DD8000730BA001030B8000730BB000830B9003F
:100DE800A0308A01462083162D0883128A014620E6
:100DF80083162C0883128A0146208A01152083163F
:100E0800C100113083128A010F200230A900831615
:100E180041088312A400A5010E30B000B1018A0177
:100E28009F2013308A010F208316AC0A0319AD0ADC
:100E38008A110A128312031DD72E00308316AA07BF
:100E480002300318013EAB0764008A110A128312AC
:100E5800031C312FFE0A0319FF0A8316BC0A8A11E4
:100E68000A128312031DC62E8A01982D11308A0199
:100E78000F2041308A010F2064308A010F2064302E
:100E88008A010F2072308A010F203A308A010F2020
:100E98000430A9007E08A4007F08A5000E30B00029
:100EA800B1018A019F200430A90083162A08831201
:100EB800A40083162B088312A5000E30B000B101E0
:100EC8008A019F200A308A010F200D308A010F20E5
:100ED80013308A010F2083160130BC00831264008E
:100EE80083163C083B028A150A128312031C042845
:100EF8008A01322383162E08AC002F08AD00831216
:100F080083162C088312A00083162D088312A100D3
:100F1800831631088312A3008316300883128A01CE
:100F280057218A110A12031DED2F0730BA0010301D
:100F3800B8000730BB000830B900A0308A0146204D
:100F480083162D0883128A01462083162C088312E3
:100F58008A0146208A0115208316C10064004108D1
:100F68000A3C8A110A1283120319D92F64008316C6
:100F780041080D3C8A110A1283120319D92F8316CE
:100F880041088312A0007E308A015521B2008316E1
:100F980041088312A00020308A015A21B400320887
:100FA80034048A110A12031DE42F11308A010F201C
:100FB8008316410883128A010F2013308A010F20FB
:100FC8008316AC0A0319AD0A8A110A128312031D8B
:100FD800842F00308316AA0702300318013EAB079E
:100FE80064008A110A128312031CFD2FFE0A0319DA
:100FF800FF0A8316BC0A8A110A128312031D732F73
:101008008A01982D83160130BC0083126400831670
:101018003C083B028A150A128312031C7C2883169B
:10102800AC01AD010130C60083126400093083169B
:1010380046028A150A1283120318632811308A019E
:101048000F204030A9000530B000B101A5013C30A7
:101058008A018F2013308A010F2013308A010F2054
:1010680013308A010F2013308A010F200730BA008D
:101078001030B8000730BB000830B900A0308A0132
:10108800462083162D0883128A01462083162C08D1
:1010980083128A0146204030A900A5013C308A010C
:1010A8002E2005308A011C2140308316AC07031816
:1010B800AD0AC60A8A150A128312031D19288A0165
:1010C800852200308316AA0702300318013EAB07B9
:1010D80064008A150A128312031C7528FE0A031974
:1010E800FF0A8316BC0A8A150A128312031D0A28EE
:1010F80011308A010F2044308A010F2061308A01A3
:101108000F2074308A010F2061308A010F202030AF
:101118008A010F2057308A010F2072308A010F2070
:1011280069308A010F2074308A010F2074308A01D7
:101138000F2065308A010F206E308A010F2013308E
:101148008A010F208A01982D8A01982D8A01982DED
:0C1158008A01982D63008A150A12AE2847
:02400E003D3D36
:00000001FF
